:020000040000FA
:02000000C52811
:08000800BB00030EBC000A0856
:10001000BD008A01831264009D3081070B11F2201C
:10002000B50B1F283230B500B715AA0303193714D2
:10003000371E1F28BE0B1F28BF0B1F28B9213D08E4
:100040008A003C0E8300BB0E3B0E09003D20B71D0D
:100050002628B711051E3428360A03193228FC3E1B
:100060000318B714B6012628360A03192628B60045
:10007000803A06300319A00026288A01200882074A
:1000800048285B286D287528802891289D28BD2840
:10009000A00A300854213713B7134321B818542845
:1000A0002B1BB717292108002B1F08007F21031CD9
:1000B000371729210800B71C6528B7100330A000A6
:1000C0000430BF00BE0137160800371C08002B089B
:1000D0001F39031D2929A00A0800A00A381D08009D
:1000E000432129210130A0000800A00AB818080007
:1000F000B71F08004321B71337170130A0000800CD
:10010000A001B8188928B00A30082F060319B001D9
:1001100008007F212C05B0002F0830020318892821
:100120000800A8013808A700B71C0800B710031082
:100130000130381D380DB80008000730371D053074
:10014000A000B7100430B706FF30B600B81D080095
:100150008B120B118B136400810183160F30810009
:1001600083128601B60163006400051AB228B60A3C
:100170003608023A031DB328C528A801A701A0012B
:100180000430BF00BE0137160800640086018316E4
:1001900010308500860100308100831220308400F9
:1001A00042308001840A0406031DD0289D3081005E
:1001B0003230B500FF3054212F03BB00AC010830B2
:1001C000BB0DAC08031D0314AC0DFF3E031DE0285E
:1001D000B0011F30A9008D210130A0000B118B163A
:1001E0008B17262822082305240525052605A104AA
:1001F000210886002508240523052205A6062408D3
:1002000023052205A50623082205A4062208A30625
:10021000A209A90B08001F30A900A1012808A2000B
:100220002708A5002805A300A400A6000800B20026
:10023000B20DB30CB20DB30CB20DB30CB20DB30CC6
:10024000B20DB30CB20DB30CB20DB30CB20D330C36
:1002500008004D218A01AA003710013E03193D29EB
:100260004D218A01371B1721B4004D218A01371B0C
:100270001721A7003408A800080048214D218A0151
:10028000AB033714080048214D218A01AB00080058
:100290002E08BA002D08B90008003A088A0039086B
:1002A000B90A0319BA0A8200B0007321B008031911
:1002B0000800AE00B10178218A01013E03197129BD
:1002C000033003190230AD070318AE0A78218A0102
:1002D000013E031D6229310AB1003006031D5B296E
:1002E00008003108AF00D930AD000130AE00080081
:1002F0002E088A002D08AD0A0319AE0A82004108B3
:1003000042040319C2090310C10DC20D031C8B293D
:10031000A130C106C206420808000301B0212F0225
:100320004008031C0301B000542143210130B021D7
:100330000739C000B8000301C00C0318013EC00C0F
:100340000318013EC00C0318013EFF3E0319AA2901
:100350000130B8000230B021C0390138B7000800C0
:100360008312890083160814831208088312C000C0
:1003700008000301C7213008CB210130C72138080C
:10038000CB210230C7213708CB2137120800831256
:1003900089008312080083128800831608155530DF
:1003A0008900AA308900881464008818D42983122F
:1003B00008000534083481340034083442340034F1
:1003C00008342434003408341834003408349934A0
:1003D000003408345A34003408343C3400340834CF
:1003E0000034183408340034183408348134183494
:1003F0000834423418340834243418340834183497
:10040000183408349934183408345A3418340834F9
:100410003C34183408341834183408343C343C3430
:1004200007347E347E340634FF34FF340834E73436
:10043000FF340A34DB34E7340A34A534C3340A34D5
:10044000423481340C3481340034FF344834053470
:10045000E0344034053470342034053438341034FA
:1004600005341C34083405340E34043405340734A0
:1004700002340534833401340534C1344034FF344C
:1004800048340334E03440340334703420340334CB
:100490003834103403341C34083403340E34043438
:1004A0000334073402340334833401340334C13455
:1004B0004034FF34483402348034803402344034D1
:1004C00040340234203420340234103410340234E6
:1004D000083408340234043404340234023402345C
:1004E0000234013401340234803480340234403424
:1004F000C0340234A0346034023450343034053413
:1005000028341834073414340C3409340A340634CB
:100510000B34053403340C34023401340E3401340A
:100520000034FF34433401348034803401344034A7
:100530004034013420342034013410341034013478
:1005400008340834013404340434013402340234ED
:1005500001340134013403340234033404340534E7
:10056000063405340B340C3406341734183407348D
:100570002E34303408345C3460340934B834C03438
:100580000A34603480340B34803400340C3400344A
:100590000034FF3448340834823481340834413420
:1005A000C0340834A0346034083450343034083453
:1005B00028341834083414340C3408340A3406341B
:1005C000083405340334FF340A3408346634003404
:1005D00008349934663408346634FF340834993466
:1005E000FF34083466349934083499340034FF34C5
:1005F0000E340734813400340734413482340734F4
:10060000A534C33407345A34E7340734A5347E3470
:1006100007345A343C34073424341834073418343B
:100620000034073400340034FF340A340834003412
:10063000CC3408340034663408340034333408349D
:1006400000349934FF3444346434FF3400341434B7
:100650007F3480341434FF3480340234FF34403427
:100660000234FF3420340234FF3410340234FF34B7
:1006700008340234FF3404340234FF3402340234C8
:10068000FF3401340234FF3400340234FF34803448
:100690000234FF3440340234FF3420340234FF3457
:1006A00010340234FF3408340234FF34043402348A
:1006B000FF3402340234FF340134FF34043407348D
:1006C000DB343C340734B734783407346F34F034D7
:1006D0000734DF34603407346F34F0340734B73410
:1006E00078340734ED341E340734F6340F340734CD
:1006F000FB3407340734F6340F340734ED341E343A
:10070000FF3404340734FF34803407347F34C0347A
:100710000734BF3460340734DF3430340734EF3407
:1007200018340734F7340C340734FB3406340734F8
:10073000FD3403340734FF3401340734FE3403340A
:100740000734FD3406340734FB340C340734F734F3
:1007500018340734EF3430340734DF34603407346E
:10076000BF34C034FF3406340734813400340734D6
:10077000423400340734243400340734183400344D
:1007800007349934003407345A34003407343C3485
:1007900000340734003418340734813418340734F3
:1007A00042341834073424341834093418341834D3
:1007B000093400341834093418340034093400344E
:1007C0001834093418341834033424343C340434D1
:1007D0005A3466340534A534C33406344234813483
:1007E000073481340034073400340034FF34FF34DC
:02400E00F63F7B
:10420000000001000000500057004D0020004C004D
:104210004500440020004300680061007300650011
:1042200072002000560031002E0030002E003700B2
:0242300020006C
:00000001FF
